:020000020000FC
:020000000EC030
:02000600E1C057
:10001C0039C00FEF01BB0FEF02BB00E004BB0EE3D6
:10002C0005BB0FEF07BB00E008BB0FE50DBF04E0FD
:10003C000EBF61E071E080E090E0A0E0B0E0E1E0B4
:10004C00C0E0D0E0F0E000E00093630000936400B7
:10005C000FEC0093660001D30BE005BD0DE403BD6E
:10006C0000E809BF00E007B900E905BF00E808B9DE
:10007C000BE006B978948895FBCF0BE806B9789419
:10008C008895089504B115B1800F911F7A9511F4DC
:10009C0070E401D0189500E110E0800F911F969547
:1000AC008795969587959695879596958795969528
:1000BC008795EC01C7D1B695A795009161001AE020
:1000CC00019F80010A1B1B0BD11720F01D1718F084
:1000DC000C1708F0FF7D009161001AE0019F800170
:1000EC000A0F1B1F1D1720F0D11718F0C01708F0AE
:1000FC00F062009160001AE0019F80010A1B1B0B4B
:10010C00D11720F01D1718F00C1708F0F0610091B2
:10011C0060001AE0019F80010A0F1B1F1D1720F0C1
:10012C00D11718F0C01708F0FF7E0091660013B3CA
:10013C0012FF0F7D11FF0F7E00936600F0230895D0
:10014C00B73018F0AE3F08F033C0B03019F4A0301F
:10015C0009F42EC020E030E040E050E0B23020F452
:10016C00B13028F0A43F18F0A45FB14007C004EFF1
:10017C0011E00A1B1B0BA02FB12F50E8B43020F458
:10018C00B33030F0A83E20F0A85EB3405395F6CFC4
:10019C00A43618F4B13008F404C0A456B04043950A
:1001AC00F7CFAA3018F0AA503395FBCF2A2F04C0F2
:1001BC002AE03AE04AE050E0A0E0B0E008956A9509
:1001CC0009F464E001D01895F8BB643031F0633069
:1001DC0061F06230B9F06130E9F04FDF022FA2D14B
:1001EC0002BB01E00F2B08BB089532D0032F9AD12C
:1001FC00E23019F0E33009F00F7702BB02E00F2B6D
:10020C0008BB089513D0042F8DD102BB04E00F2B33
:10021C0008BB0895CCD0052F003011F083D101C05C
:10022C000FEF02BB08E00F2B08BB0895FF73009182
:10023C00660004FF05C0E33019F074FFF4FFF064AE
:10024C0005FF05C0E23019F074FFF5FFF068089562
:10025C00E13031F0E23039F0E33069F0E43099F01C
:10026C00DE016EDF0895009160001AE0019FD0015D
:10027C0067DF22E80895009161001AE0019FD00128
:10028C005FDF22E80895DED004EF11E0A00FB11F6C
:10029C0057DF51E8403009F442E80895E13031F07D
:1002AC00E23081F0E330F1F0E43029F100916600A6
:1002BC0004FF02C00F7E03C013B311FD0061009355
:1002CC0066000895009160000395093C08F008EC65
:1002DC000093600010916100011718F003950093D2
:1002EC00610008950091610003950A3C08F009EC47
:1002FC000093610008950091620003950A3108F0A3
:10030C0009E1009362000895E13031F0E23081F0B0
:10031C00E330B9F0E43029F10091660005FF02C02A
:10032C000F7D03C013B312FD0062009366000895A5
:10033C00009160000A95093008F409E00093600010
:10034C000895009161000A950A3008F40AE00093C0
:10035C00610010916000101718F00A95009360006E
:10036C000895009162000A950A3108F000E00093AC
:10037C0062000895EA9509F4E3E00091660005FD3A
:10038C0003C0E33009F4EA950091660004FD03C054
:10039C00E23009F4EA952CD10895E13009F07EDFC2
:1003AC000895E13009F0B0DF0895E4E0089500917C
:1003BC006400003019F00A950093640010916300FA
:1003CC0003B3087300936300101781F0109164005D
:1003DC00103061F403FF05C004FF05C005FF05C024
:1003EC0005C05CDF03C090DF01C0C4DF15E003FF74
:1003FC001093640004FF1093640005FF10936400D5
:10040C00083329F010916500139510936500109135
:10041C006400103019F410E0109365001091650021
:10042C00143679F41FE51093650003FF05C004FF33
:10043C0005C005FF05C005C0B0DF03C0B2DF01C0B9
:10044C00B4DF0895B0E000916200003091F101300A
:10045C0091F1023091F1033091F1043091F10530BA
:10046C0091F1063091F1073091F1083091F109309A
:10047C0091F10A3091F10B3091F10C3091F10D307A
:10048C0091F10E3091F10F3091F1003191F1013178
:10049C0091F1023191F1033191F1043191F1053176
:1004AC0091F1063199F10731A1F10831A9F1093126
:1004BC00B1F1A2E00895A4E00895A6E00895A8E0A3
:1004CC000895AAE00895ACE00895AEE00895A0E187
:1004DC000895A4E10895A8E10895AEE10895A8E275
:1004EC000895A2E30895ACE30895A0E50895A4E669
:1004FC000895A8E70895ACE80895A0EA0895A8EC3B
:10050C000895A0EF0895ACE2B1E00895A0E9B1E040
:10051C000895A4EFB1E00895A8E5B2E00895A0E233
:10052C00B3E008950030D1F00130D1F00230D1F0B9
:10053C000330D1F00430D1F00530D1F00630D1F0D9
:10054C000730D1F00830D1F00930D1F00038D1F0BB
:10055C000138D1F00238D1F007EF089500EC08957E
:10056C0009EF089504EA089500EB089509E9089548
:10057C0002E9089502E8089508EF089500E8089547
:10058C0000E908950FEB089509E808950FEF089519
:10059C00E199FECF00E00EBB00E00FBB00916100C3
:1005AC000DBBE29AE19A0895E199FECF01E00EBBF2
:1005BC0000E00FBB009160000DBBE29AE19A089538
:1005CC00E199FECF02E00EBB00E00FBB0091620090
:1005DC000DBBE29AE19A0895E199FECF03E00EBBC0
:1005EC0000E00FBB009166000DBBE29AE19A089502
:1005FC00E199FECF00E00EBB00E00FBBE09A0DB31B
:10060C0010916100011709F0C3DFE199FECF01E001
:10061C000EBB00E00FBBE09A0DB310916000011708
:10062C0009F0C2DFE199FECF02E00EBB00E00FBB88
:10063C00E09A0DB310916200011709F0C1DFE19946
:10064C00FECF03E00EBB00E00FBBE09A0DB31091A0
:10065C006600011709F0C0DF0895E199FECF00E0B4
:10066C000EBB00E00FBBE09A0DB30A3C08F00BE4A4
:10067C0000936100E199FECF01E00EBB00E00FBBDF
:10068C00E09A0DB3093C08F006E400936000E19990
:10069C00FECF02E00EBB00E00FBBE09A0DB30A31B7
:1006AC0008F004E000936200E199FECF03E00EBB7A
:1006BC0000E00FBBE09A0DB3102F1F7C1F3C09F01C
:0806CC000FEC00936600089595
:00000001FF
